:020000040800F2
:10000000A80A0020A9010008A5050008810500082C
:1000100000000000000000000000000000000000E0
:10002000000000000000000000000000A90500081A
:100030000000000000000000A7050008F905000806
:10004000BB010008BB010008BB010008BB010008A0
:10005000BB010008BB010008BB010008BB01000890
:1000600000000000BB010008BB010008BB01000844
:10007000BB010008BB010008BB0100080000000034
:10008000BB010008BB01000800000000AD0600082D
:10009000DD060008BB010008BB010008BB01000829
:1000A000BB010008BB010008BB01000841070008B4
:1000B000BB0100080000000000000000000000007C
:1000C000BB01000800000000BB01000800F002F8BE
:1000D00000F03EF80CA030C8083824182D18671E10
:1000E000A246AB4654465D46AC4201D100F030F822
:1000F0007E460F3EB6460FCC0126334200D0FB1A97
:100100003343A246AB461847F836000018370000C4
:10011000103A02D378C878C1FAD8520701D330C850
:1001200030C101D504680C60704700000023002432
:1001300000250026103A01D378C1FBD8520700D31E
:1001400030C100D50B6070471FB51FBD10B510BD85
:1001500000F0A5F91146FFF7F7FF01F09BFF00F053
:10016000BDF903B4FFF7F2FF03BC00F08BF9000008
:1001700070B505460C46164602E00FCC0FC5103E82
:10018000102EFAD2082E02D303CC03C5083E042E4B
:1001900007D301CC01C5361F03E021782970641C08
:1001A0006D1C761EF9D270BD07488047074800478E
:1001B000FEE7FEE7FEE7FEE7FEE7FEE70448054947
:1001C000054A064B7047000001060008CD000008F4
:1001D000A8020020A80A0020A8060020A8060020E7
:1001E0000EB5044615460E4612A000F085F82046CE
:1001F00000F082F815A000F07FF8304600F07CF89F
:1002000014A000F079F86C460020E0720A20A07279
:100210000A3407E00A21284600F082F8303105460A
:10022000641E2170002DF5DC204600F065F800F01A
:1002300059F800002A2A2A20617373657274696F65
:100240006E206661696C65643A2000002C20666946
:100250006C6520002C206C696E652000F8B5042ABE
:100260002CD3830712D00B78491C0370401C521EFC
:1002700083070BD00B78491C0370401C521E830768
:1002800004D00B78491C0370401C521E8B079B0F37
:1002900005D0C91ADF002023DE1B08C90AE0FFF7DA
:1002A00067FFF8BD1D4608C9FD401C46B4402C43FD
:1002B00010C0121F042AF5D2F308C91A521EF0D436
:1002C0000B78491C0370401C521EEAD40B78491C61
:1002D0000370401C012AE4D409780170F8BD70470E
:1002E0007047704710B5002000F0D2F8FFF72EFFDE
:1002F000012000F0C7F810BD10B5044602E0641CF0
:1003000000F0BAF820780028F9D110BD00220309C6
:100310008B422CD3030A8B4211D300239C464EE020
:1003200003460B433CD4002243088B4231D30309DC
:100330008B421CD3030A8B4201D394463FE0C3098E
:100340008B4201D3CB01C01A524183098B4201D3A6
:100350008B01C01A524143098B4201D34B01C01A91
:10036000524103098B4201D30B01C01A5241C30809
:100370008B4201D3CB00C01A524183088B4201D378
:100380008B00C01A524143088B4201D34B00C01A64
:100390005241411A00D201465241104670475DE079
:1003A000CA0F00D04942031000D3404253409C463C
:1003B000002203098B422DD3030A8B4212D38901F9
:1003C000FC2212BA030A8B420CD3890192118B4290
:1003D00008D3890192118B4204D389013AD092113A
:1003E00000E08909C3098B4201D3CB01C01A5241F5
:1003F00083098B4201D38B01C01A524143098B42BE
:1004000001D34B01C01A524103098B4201D30B01A6
:10041000C01A5241C3088B4201D3CB00C01A5241CB
:1004200083088B4201D38B00C01A5241D9D24308B2
:100430008B4201D34B00C01A5241411A00D20146EF
:100440005241104663465B1001D34042002B00D559
:100450004942704763465B1000D3404201B50549ED
:10046000002802DC491C084000E00846C046C0469F
:1004700002BD00BFFFFFFF7F08B56946087003207B
:10048000ABBE08BD01491820ABBEFEE72600020046
:1004900010B500F031F800F029F810BD704775462E
:1004A00000F042F8AE46050069465346C008C00059
:1004B000854618B020B5FFF781FE60BCB646002621
:1004C0000027C0C5C0C5C0C5C0C5C0C5C0C5C0C562
:1004D000C0C5403D490849008D46704710B50446E7
:1004E000C046C0462046FFF73CFE10BD10B50028B0
:1004F00001D0FFF7C7FF10BD10B5002102A000F02A
:1005000017F8012010BD0000534947414252543AA8
:100510002041626E6F726D616C207465726D696EE0
:100520006174696F6E0000000048704798000020F9
:1005300070B505460C460A2000E06D1CFFF79CFFD5
:10054000002D06D028780028F7D102E0641CFFF7C0
:1005500093FF002C02D020780028F7D10A20FFF763
:100560008BFF70BD81B00090009874490860FFE770
:100570007248006808B1FFE7FAE701B07047C0466B
:10058000FFE7FEE780B50648006840F2E831B0FBBF
:10059000F1F000F00BF810B1FFE7FFE7FEE780BDD8
:1005A00000000020704770477047000080B584B09D
:1005B00002900298401E000E18B1FFE70120039040
:1005C00011E00298401E0949086000200190C043D4
:1005D000032100F051F9019805490860054A0721F7
:1005E00011600390FFE7039804B080BD14E000E0C1
:1005F00018E000E010E000E080B500F095F880BD64
:1006000080B582B020490868012210430860FFE7E6
:100610001D4800688007002801D4FFE7F8E71B4960
:1006200008681B4A1040086008681A4A10400860B1
:1006300015490868184A10400860184908680F22D0
:10064000904308601649086840F20312904308601E
:100650000868012200921304984308600868D307D1
:10066000984308600F490868904308600E490020CD
:100670000190086002F01AF800980199C00601F094
:1006800073FD02B080BDC04600100240041002405D
:100690000C00FF08FFFFC277FFFFF2FE2C100240A4
:1006A00030100240341002400810024080B582B081
:1006B0000948012102F04EF960B1FFE706480190B8
:1006C000012102F03DF90198002102F01BF801F030
:1006D000F1FDFFE702B080BD0020004080B50E486C
:1006E000012102F037F9012805D1FFE70A4801216D
:1006F00002F026F9FFE709480168491C016000681B
:100700000749884207D1FFE70449002008600549EE
:1007100001200870FFE780BD004001402401002057
:10072000B80B0000280100200448006828B1FFE74A
:1007300002490868401E0860FFE770475401002026
:1007400080B51B481B4902F073FA38B1FFE701F08E
:10075000B9FD1748174902F04BFAFFE7144816494C
:1007600002F006FA012807D1FFE71148124902F00A
:10077000F0F901F0A7FDFFE70D48104902F058FA23
:1007800038B1FFE701F0A6FD09480C4902F030FA44
:10079000FFE707480A4902F04BFA38B1FFE701F0DA
:1007A00099FD0348064902F023FAFFE780BDC046E1
:1007B0000038014005000507030700000700070790
:1007C0000600060781B0014668460170007840B215
:1007D00000280DD4FFE76846007841B21F200A4682
:1007E00002400120904049098900024A8850FFE7F1
:1007F00001B0704700E100E070B582B0024601A888
:1008000002700091007840B2002817D4FFE701A9D8
:10081000087840B20322D3431840384A80580978F8
:1008200049B28C07E50EFF24AC40A043009CA40114
:10083000E4B2AC402043194088501AE001A908787E
:100840000F24204008380322D34318402A4A8058F6
:10085000097849B28D07EE0EFF25B540A843009DEB
:10086000AD01EDB2B5402843214008391940885008
:10087000FFE702B070BDC04670B582B0024601A865
:1008800002700091007840B2002817D4FFE701A958
:10089000087840B20322D3431840184A8058097898
:1008A00049B28C07E50EFF24AC40A043009CA40194
:1008B000E4B2AC402043194088501AE001A90878FE
:1008C0000F24204008380322D34318400A4A805896
:1008D000097849B28D07EE0EFF25B540A843009D6B
:1008E000AD01EDB2B5402843214008391940885088
:1008F000FFE702B070BDC0461CED00E000E400E080
:1009000080B584B0039002A8017001A9FF2008708F
:10091000039800285CD0FFE702A80078401E0090F2
:10092000052853D800998A0001A080188746C04640
:1009300000F00AB800F013B800F01CB800F025B8B9
:1009400000F02EB800F037B80920C006012101F0F0
:100950009BFA0399088001A90020087037E009205C
:10096000C006022101F090FA0399088001A9002035
:1009700008702CE00920C006042101F085FA0399D3
:10098000088001A90020087021E00920C006082184
:1009900001F07AFA0399088001A90020087016E096
:1009A0000920C006102101F06FFA0399088001A9FF
:1009B000002008700BE00920C006202101F064FA35
:1009C0000399088001A90020087000E0FFE7FFE715
:1009D00001A8007804B080BD80B584B0224801F041
:1009E000BDFD0920C0060090002102910123039360
:1009F0001A4601F05EFA00980299039A022301F068
:100A000058FA00980299039A042301F052FA0098C8
:100A10000299039A082301F04CFA00980299039A6C
:100A2000102301F046FA00980299039A202301F05E
:100A300040FA0E4801F092FD0299039A264801906F
:100A400044F2000301F035FA01980299039A42F248
:100A5000000301F02EFA01980299039A41F2000373
:100A600001F027FA04B080BD110500001205000056
:100A700080B582B001A900200870174844F2000137
:100A800001F002FA30B1FFE701980121084301A902
:100A90000870FFE7104842F2000101F0F5F930B1AB
:100AA000FFE701980221084301A90870FFE70A48FF
:100AB00041F2000101F0E8F930B1FFE701980421AB
:100AC000084301A90870FFE701980721814301A8A5
:100AD0000170007802B080BD0004004810B586B0F7
:100AE00005AC207004A80170039202AA137001AB38
:100AF000002119700F4B0A2119700078039913789F
:100B0000072202F047FB012804D0FFE701A90320D8
:100B100008700AE0084802F0BDFB012804D0FFE796
:100B200001A903200870FFE7FFE701A8007806B0DD
:100B300010BDC04659010020204E000080B584B091
:100B400003900291019269460020087017480088BE
:100B5000FF2801DCFFE704E0154816499C22FFF757
:100B60003FFB12480088032817DBFFE73148006885
:100B70000E49098801F07FFB78B9FFE72D4801682D
:100B80000978039A117009490988891E019A118010
:100B90000068401C0299086003E06946052008705F
:100BA000FFE76846007804B080BDC0467E020020A2
:100BB00065370008E6370008B0B586B005AB187099
:100BC000049103A8028002A900200870224800783E
:100BD00018BBFFE70498411E14480160144D012121
:100BE00000912980059902681170039A2988891853
:100BF00029800068298801F03EFB009901AA107045
:100C000001980C4A12682B885C1C2C80D0540A482E
:100C10000170002002F09AF803E002A90520087094
:100C2000FFE702A8007806B0B0BDC046380100203A
:100C3000A2020020080000202001002080B582B020
:100C400001200021019102F081F801980249087009
:100C500002F084FA02B080BD1E01002080B50021A0
:100C6000084602F073F802F0B1F880BD80B582B09A
:100C700001A9002008700A480078012807D1FFE781
:100C800008480068804706490020087003E001A971
:100C900006200870FFE701A8007802B080BDC046BA
:100CA000040000204001002080B588B00790069124
:100CB00001A9002008700698008805286BD1FFE77D
:100CC00007984078000205A908800798827805985F
:100CD000104308800598401C08800798C0780102DE
:100CE00004A8018007990A790499114301800088BA
:100CF00001284BDBFFE704A800886A49884245DCED
:100D0000FFE7079802900699002008800299481C86
:100D100002900120087006990888401C088004A8E9
:100D20000078400738B1FFE704A80088C008401CDD
:100D300003A9087004E00498C00803A90870FFE73D
:100D4000039802994A1C0292087006990888401C70
:100D50000880029805A9098804AA1288002300F0D7
:100D600005FE014668460170007838B1FFE7684625
:100D7000007801F009FA01A9087006E003A80278DA
:100D80000699088880180880FFE703E001A903207E
:100D90000870FFE703E001A903200870FFE701A83E
:100DA000007808B080BDC04680B588B00790069135
:100DB00001A9002008700698008805286AD1FFE77D
:100DC00007984078000205A908800798827805985E
:100DD000104308800598401C08800798C0780102DD
:100DE00004A8018007990A790499114301800088B9
:100DF00001284ADBFFE704A800882A49884244DC2E
:100E0000FFE7079802900699002008800299481C85
:100E100002900220087006990888401C088004A8E7
:100E20000078400738B1FFE704A80088C008401CDC
:100E300003A9087004E00498C00803A90870FFE73C
:100E4000039802994A1C0292087006990888401C6F
:100E50000880029805A9098804AA128800F03CFEBF
:100E6000014668460170007838B1FFE768460078AF
:100E700001F08AF901A9087006E003A80278069932
:100E8000088880180880FFE703E001A903200870A4
:100E9000FFE703E001A903200870FFE701A800783D
:100EA00008B080BDCF07000080B588B007900691DC
:100EB00002A90020087006980088052857D1FFE78E
:100EC00007984078000205A908800798827805985D
:100ED000104308800598401C08800798C0780102DC
:100EE00004A801800799097901800088012839DB6D
:100EF000FFE704A800887D2834DCFFE7079803900B
:100F00000698002303800399481C0390032008706F
:100F100006990888401C08800498400003994A1CE0
:100F20000392087006990888401C0880039805A958
:100F3000098804AA128800F04BFE014601A801703E
:100F4000007838B1FFE701A8007801F01DF902A987
:100F5000087006E004984200069908888018088006
:100F6000FFE703E002A903200870FFE703E002A9FE
:100F700003200870FFE702A8007808B080BD80B5A4
:100F800088B00790069102A9002008700698008892
:100F9000052859D1FFE707984078000205A9088085
:100FA000079882780598104308800598401C0880AF
:100FB0000798C078010204A8018007990A7904996A
:100FC000114301800088012839DBFFE704A800886D
:100FD0007C2834DCFFE707980390069900200880FE
:100FE0000399481C03900420087006990888401C47
:100FF00008800498400003994A1C039208700699DF
:101000000888401C0880039805A9098804AA12884A
:1010100000F066FE014601A80170007838B1FFE7D4
:1010200001A8007801F0B0F802A9087006E0049861
:1010300042000699088880180880FFE703E002A9AB
:1010400003200870FFE703E002A903200870FFE710
:1010500002A8007808B080BD80B58AB009900891D8
:1010600001A900200870089800880A2800DA99E091
:1010700009984078000207A90880099882780798A3
:10108000104308800798401C08800998C078010226
:1010900006A8018009990A790699114301800999E6
:1010A0004979090205AA118009998B790599194393
:1010B00011800599491C11800999C979090204AA6E
:1010C000118009990B7A0499194311800999497A79
:1010D00003AA1170008801285FDBFFE706A80088DB
:1010E0007D285ADCFFE704A80088012855DBFFE7CC
:1010F00004A80088792850DCFFE704A80088410094
:1011000003A80078884248D1FFE709980A3005A96A
:10111000098804AA1288012300F05AFD0146684696
:101120000170007868BBFFE70998029008980023D7
:1011300003800299481C02901720087008990888BB
:10114000401C08800698400002994A1C02920870D0
:1011500008990888401C0880029807A9098806AAEF
:10116000128800F035FD014668460170007838B9F4
:10117000FFE7069842000899088880180880FFE772
:10118000FFE76846007838B1FFE76846007800F06E
:10119000FBFF01A90870FFE703E001A90320087025
:1011A000FFE7FFE701A800780AB080BD80B584B0F2
:1011B000039002910398401C064901910A88064950
:1011C000FFF74CF801980088401C02990880002025
:1011D00004B080BD7A0200205A01002080B586B09C
:1011E0000590049101A90020087004980088052842
:1011F00044D1FFE705984078000203A908800598CC
:1012000082780398104308800398401C0880059852
:10121000007970BBFFE70598C078FF2804D0FFE78E
:101220000598C07828BBFFE702A900204870059800
:10123000C078FF2804D1FFE702A90120087003E06D
:1012400002A900200870FFE703A8018802A8012373
:101250001A4600F08BFB014668460170007838B1F1
:10126000FFE76846007800F08FFF01A90870FFE7EC
:1012700003E001A903200870FFE703E001A90320B0
:101280000870FFE701A8007806B080BD80B586B081
:101290000590049102A90020087004980088052890
:1012A00022D1FFE705984078000203A9088005983D
:1012B00082780398104308800398401C08800598A2
:1012C000C01C098801231A4600F082FC014601A8CF
:1012D0000170007838B1FFE701A8007800F054FFF2
:1012E00002A90870FFE703E002A903200870FFE7E6
:1012F00002A8007806B080BD80B588B0079006913E
:1013000001A9002008700698008806285EDBFFE728
:1013100007984078000205A9088007988278059808
:10132000104308800598401C08800798C078010287
:1013300004A8018007990A7904991143018007994B
:10134000497903AA11700088400738B1FFE704A863
:101350000088C008401C02A9087004E00498C00876
:1013600002A90870FFE704A80088012829DBFFE72D
:1013700004A8008840F2B071884222DCFFE702A88E
:10138000007803A9097888421BD1FFE70798801DE0
:1013900005A9098804AA1288012300F0E7FA01468A
:1013A00068460170007838B1FFE76846007800F0C1
:1013B000EBFE01A9087003E0069905200880FFE70D
:1013C00003E001A903200870FFE703E001A903205F
:1013D0000870FFE701A8007808B080BD80B588B02C
:1013E0000790069102A90020087006980088062838
:1013F0004CDBFFE707984078000205A908800798B2
:1014000082780598104308800598401C088007984A
:10141000C078010204A8018007990A790499114350
:1014200001800799497903AA11700088012828DBF7
:10143000FFE704A80088782823DCFFE703A80078EA
:1014400004994900C9B288421BD1FFE70798801D63
:1014500005A9098804AA1288012300F0B9FB0146F6
:1014600001A80170007838B1FFE701A8007800F00A
:101470008BFE02A9087003E0069905200880FFE7AB
:1014800003E002A903200870FFE703E002A903209C
:101490000870FFE702A8007808B080BDB0B588B03A
:1014A0000C460C9907AD287006A8047005AC227094
:1014B000049303AA117002AA00211170007850B1A0
:1014C000FFE706A80078012805DBFFE706A80078FB
:1014D000F82804DBFFE702A9022008706CE00698F8
:1014E000AD49087007A80078019020B1FFE7019886
:1014F000012824D047E032493E48086032493E483E
:101500000860A4493D480860A4493D480860324944
:101510000020086031493B48086032493A48086079
:1015200032493A4808609C48007805A90978049A2D
:1015300003AB1B7800F034F902A9087027E02049BA
:1015400020480860204921480860924920480860E6
:101550009249204808602049002008601F4920481F
:1015600008602049204808602049214808608A48CE
:10157000007805A90978049A03AB1B78FFF7AEFA47
:1015800002A9087003E002A902200870FFE702A880
:10159000007880B9FFE701F0DBFD20B9FFE702A981
:1015A0000320087006E00798794908707149012006
:1015B0000870FFE7FFE7FFE702A8007808B0B0BDBA
:1015C000400100203D0C0008440100205D0C000893
:1015D000B90B00083D0B00083C0100204801002029
:1015E000292E00084C010020D52F000850010020B2
:1015F0008D2F0008451900085D190008991800088A
:1016000019180008F932000829340008A933000825
:10161000B0B586B003A9002008705648007820B104
:10162000FFE705A906200870A0E002A801F078FDF8
:10163000012800D096E002A800780190032800D984
:101640008FE001998A0001A08018874600F006B853
:1016500000F005B800F020B800F082B881E04F48F3
:1016600003684A484449484A9847014603A801701C
:10167000007880B9FFE745480078474909788842F3
:1016800004D0FFE74148007820B9FFE7022001F0CD
:1016900065FDFFE7FFE764E03748006800783749F9
:1016A000087037490120087000200490FFE7049873
:1016B0000F2822DCFFE70498C1003248405C08B9DB
:1016C000FFE71AE00498C1002E48405C2B490978D6
:1016D00088420CD1FFE70498C1002A4840184268AC
:1016E00025480068284990472549087005E0FFE72C
:1016F000FFE70498401C0490D9E72448007870B3B1
:10170000FFE71F480078A8B1FFE71F4C00202080AA
:101710001A4800788021084317490A6823885D1C0D
:101720002580D0541648007809682288531C2380ED
:101730008854FFE716480078012804D1FFE701200C
:1017400008B9FFE7FFE713480368134800780A4920
:1017500009680D4A1288984703A90870FFE700E05E
:10176000FFE7FFE705A900200870FFE705A800785C
:1017700006B0B0BD040000201401002011010020BB
:1017800010010020140000201A0100201801002080
:101790000F01002030010020580100202C01002002
:1017A00010B586B005AC207004A80170039202AA9F
:1017B000137001AB00211970007803991378082287
:1017C00001F0E8FC012804D0FFE701A9032008701C
:1017D0001AE003980E49884203D3FFE723200090C4
:1017E00006E0039841000B48B0FBF1F00090FFE7E2
:1017F0006846008801F04EFD012804D0FFE701A9EA
:1018000003200870FFE7FFE701A8007806B010BDCD
:10181000014B0000A07F170080B586B005900491B1
:10182000039202A90020087001A9087017480088D7
:10183000FF2801DCFFE704E0154816499C22FEF76B
:10184000CFFC12480088042817DBFFE70F48018807
:101850003A4801F0B1F880B9FFE738480178059AB5
:1018600011700A490988C91E039A11800499401C05
:10187000086002A90120087003E001A90520087092
:10188000FFE701A8007806B080BDC0467C020020BA
:10189000653700088A370008B0B588B007AB187004
:1018A000069105A8028004A9002008702A48007843
:1018B000012837D1FFE70698411E1E4800900160BD
:1018C0001D4D01950121029129800799026811702F
:1018D000059A2988891829800068298801F06CF800
:1018E0000246009803A90A80039B2C88621C2A8068
:1018F000124A135549782B885C1C2C80D1540068FF
:10190000007801F0B9FC009B019A02991868401C0C
:1019100018601088401E108009480170002001F0F6
:1019200015FA03E004A905200870FFE704A8007871
:1019300008B0B0BD34010020A00200207A010020D0
:101940001F01002080B5044800210170012001F032
:10195000FDF901F051FA80BD1D01002080B5002184
:10196000084601F0F3F901F031FA80BD10B58EB0F0
:1019700003920A4603990D900CA802800BAA1180CD
:101980000AA90B7009AB002119701288521E530F5F
:10199000D218D208521C07AB1A8006AA117005AAE9
:1019A000117004AA11700C99491E0180008800284A
:1019B00000D585E00CA800880BA9098840180428E8
:1019C00000DD7DE00C9842490988401A08A908808A
:1019D0000AA80078029020B1FFE70298012839D0C8
:1019E0006DE0FFE707AA1088411E118088B3FFE76A
:1019F00004A90020087005A908200870FFE70BAAB9
:101A00001188481E10800020019041B1FFE705AA0F
:101A10001078411E1170411E88410190FFE7019826
:101A2000C00780B1FFE708AA1188481C1080294828
:101A3000415C04AB1878421C1A7081400698084338
:101A400006A90870DBE706980D994A1C0D920870EC
:101A5000C8E734E0FFE707AA1088411E118068B389
:101A6000FFE70D98411C0D91007806A9087005A9A3
:101A700008200870FFE70BAA1188481E108000207C
:101A8000009041B1FFE705AA1078411E1170411E78
:101A900088410090FFE70098C00770B1FFE706A9F2
:101AA00008780122104008AC23885A1C2280094A79
:101AB000D054087840080870DDE7CCE7FFE703E082
:101AC00009A901200870FFE709A800780EB010BD31
:101AD00084020020800200208BB001920A46019906
:101AE0000A9009A8028008AA118007AB002119708A
:101AF0001288521E530FD218D208521C05AB1A80FE
:101B000004AA117003AA117002AA11700999491E42
:101B10000180008840F2E83188424DDBFFE709A8E8
:101B2000008808A90988401840F2EC31884243DC5B
:101B3000FFE7099824490988401A06A90880FFE7A9
:101B400005AA1088411E1180A8B3FFE702A9002052
:101B5000087003A908200870FFE708AA1188481E2A
:101B600010800020009041B1FFE703AA1078411EC9
:101B70001170411E88410090FFE70098C007A0B196
:101B8000FFE706A801881148405C48B1FFE702A8BA
:101B90000078012181400498084304A90870FFE7F8
:101BA0000298401C02A90870D7E704980A994A1CB9
:101BB0000A920870C4E703E007A901200870FFE754
:101BC00007A800780BB070470C00002086020020A8
:101BD00010B588B0079006A8018005A90A8004A95D
:101BE0000B7003AA002111700699491E018000881C
:101BF000354988425FDBFFE706A8008805A9098808
:101C000040183249884256DCFFE706A80088304970
:101C10000988401A029002982E49086004A80078AA
:101C2000009020B1FFE70098012842D042E006A8CA
:101C30000088254988421DDBFFE706A80088234964
:101C4000884217DCFFE700F099F80190069840F60B
:101C50009801401A204A1070029841001F4840180D
:101C6000019912785200891805AA12885200FEF7CD
:101C7000F5FAFFE7FFE705A80088012818DBFFE772
:101C800002984100154841184978079A531C079358
:101C9000117002994900405A07994A1C079208702E
:101CA0000298401C02900598401E05A90880E2E7B2
:101CB00000E0FFE703E003A901200870FFE703A8A5
:101CC000007808B010BDC046980800009F080000CA
:101CD0000E000020FC000020F80000208A020020F6
:101CE00085B0049003A8018002A90A8001AA0021FE
:101CF00011700399491E0180008840F2D07188421A
:101D00002EDBFFE703A8008802A9098840181849BC
:101D1000884225DCFFE703A8008816490988401A95
:101D20000090FFE702A80088012818DBFFE7009871
:101D30004100114841184978049A531C04931170CA
:101D400000994900405A04994A1C0492087000986E
:101D5000401C00900298401E02A90880E2E703E0C0
:101D600001A901200870FFE701A8007805B07047BD
:101D7000D40700001000002098020020004870479F
:101D80000001002086B00590049103920598006A36
:101D900001900598406A009002A900200880FFE7A2
:101DA00002A8008807281DD8FFE702A80188039829
:101DB000C840C00780B1FFE702A8018889000F2250
:101DC0008A400199914301910499008880008140E3
:101DD000019808430190FFE7FFE70298401C02A921
:101DE0000880DDE702A908200880FFE702A8008834
:101DF0000F281FD8FFE702A801880398C840C00732
:101E000090B1FFE702A80188890020390F228A409B
:101E10000099914300910499008880002038814006
:101E2000009808430090FFE7FFE70298401C02A9D2
:101E30000880DBE7019805990862009805994862D7
:101E400006B0704782B001900091009801998862B5
:101E500002B0704782B001900091009801998861AA
:101E600002B0704783B0029001916846027000781A
:101E700020B1FFE701980299886103E00198029977
:101E80008862FFE703B0704783B00190009101982A
:101E900000690099084204D0FFE702A901200870F8
:101EA00003E002A900200870FFE702A8007803B051
:101EB000704787B0069005910492039306980068D6
:101EC00001900698C068009002A900200880FFE7F2
:101ED00002A800880F282BD8FFE702A801880398E2
:101EE000C840C007F0B1FFE702A8018849000322FB
:101EF00013468B40019999430191059B0188490044
:101F00008B40019919430191018849008A40009949
:101F10009143009104990088400081400098084353
:101F20000090FFE7FFE70298401C02A90880CFE776
:101F300001980699086000980699C86007B0704734
:101F400010B586B0059004A8017003920293007842
:101F5000012806D1FFE7029A0599486810434860B6
:101F600005E0029A0599486890434860FFE70598A4
:101F70008068009001A900200880FFE701A8008880
:101F80000F281DD8FFE701A801880298C840C007A4
:101F900080B1FFE701A80188490003228A40009927
:101FA00091430091039900884000814000980843C4
:101FB0000090FFE7FFE70198401C01A90880DDE7DA
:101FC00000980599886006B010BD000080B586B005
:101FD00005A908702E480078A8B3FFE70920C006BD
:101FE00040F200110122FFF73DFF00200490FFE7BF
:101FF000049805A9097888421ADAFFE70920C00683
:10200000019040F2001102910022FFF72BFF6420A3
:102010000390FEF7A7FA019802990122FFF722FF29
:102020000398FEF79FFAFFE70498401C0490DFE74F
:102030000920C00640F200110122FFF713FF1449E6
:1020400000200870FFE706B080BDC04680B584B0B0
:102050000E4800F083FA0920C006019001210022F9
:10206000039240F200130293FFF723FF0198029BB3
:1020700003990322FFF764FF01980299FFF7EAFE34
:1020800003980349087004B080BDC04611050000E4
:102090002801002080B588B0002002900790FEF74C
:1020A000AFFAFEF76FFAFEF797FCFFF7CFFF224873
:1020B000472100F0FFFAFEF7DBFC029A06A9087040
:1020C0000699403105A8017001780092E120430291
:1020D0001046FFF7E3F9FEF7C9FDFFF74FFE014693
:1020E0000298049103AA107005980002801D0499BB
:1020F000127852008852FFE7FFF78AFA03A90120FD
:102100000870FFE703A8007806280DDCFFE70498B5
:1021100003A909784A008018FEF7F2FBFFE703984D
:10212000401C03A90870EDE706A80078FFF74EFFF2
:102130001420FEF717FADFE7E703000080B584B04C
:102140000A46014603A80190017002A90A700078AE
:1021500040B20978FEF750FB0198007840B2FEF7D4
:1021600031FB04B080BD000082B001900091019865
:102170000099034A114008430249086002B07047C1
:1021800080FFFF1F08ED00E083B0014602A8017048
:102190000078009040B1FFE70098012808D0FFE7E1
:1021A0000098072808D00BE001A9002008700BE078
:1021B00001A90220087007E001A90620087003E0C9
:1021C00001A904200870FFE701A8007803B0704758
:1021D00082B00146684601700078092805DCFFE7F7
:1021E0000098303001A9087014E0684600780A2889
:1021F0000ADBFFE7684600780F2805DCFFE7009858
:10220000373001A9087005E00448054940F2D012B2
:10221000FDF7E6FF01A8007802B07047E437000838
:10222000E637000882B00146684601700078302821
:102230000ADBFFE768460078392805DCFFE70098ED
:10224000303801A9087012E06846007841280ADB9E
:10225000FFE768460078462805DCFFE70098373836
:1022600001A9087003E001A9FF200870FFE701A899
:10227000007802B0704783B0029001A801806946DF
:1022800000200870FFE701AA1088411E118048B1A4
:10229000FFE70298411C02910178009840186946B6
:1022A0000870F0E70098414268460170007803B07A
:1022B0007047000080B502480068804780BDC04676
:1022C0005001002080B502480068804780BDC046AC
:1022D0004801002080B502480068804780BDC046A4
:1022E0004C0100209CB01BA90870002001901A909E
:1022F00019901890179016901590149013901290B2
:10230000119010900F900E900D900C900B908B49A7
:102310000A918B49099108900790069105900491C4
:102320000390DF4800680C21084080081A901A9832
:10233000029040B1FFE70298012807D0FFE702981A
:10234000022806D044E08148169044E07F48169069
:1023500041E0D34801680F2292041140890C10918A
:1023600000680121C9060840C00E0F900F9801288F
:1023700004D1FFE71098113010900BE010980F284F
:1023800003D1FFE71020109003E01098801C1090FC
:10239000FFE7FFE7C2480068012109040840000C7C
:1023A0000E900E9870B1FFE7674800680F21084053
:1023B000401C0D900D996548B0FBF1F11098484311
:1023C000169004E010995F4848431690FFE702E03A
:1023D0005E481690FFE7B2480168C9B209090C913E
:1023E0000C9A07A9895C0B9116990B9AD14015910B
:1023F000016840F200721140090A0C910C9A05A97B
:10240000895C0B9115990B9AD1401491006843F6A1
:1024100000010840C00A0C900C9903A8405C0B9086
:1024200015980B99C84013901BA8007800900528B8
:1024300000D97FE000998A0001A080188746C04635
:1024400000F00AB800F00BB800F00CB800F00DB8BE
:1024500000F00EB800F040B8169817906BE0159891
:10246000179068E01498179065E01398179062E051
:102470003748006840F20011084088420FD0FFE75B
:1024800033480068012109040840884203D0FFE76F
:102490003148129002E02F481290FFE719E080487F
:1024A000006880B2800B199029480068C00F18900E
:1024B000189838B1FFE715981999491CB0FBF1F04D
:1024C000129005E013981999B0FBF1F01290FFE714
:1024D000FFE7129817902EE01D480068800718B992
:1024E000FFE71398119022E0194800680321084083
:1024F000012803D1FFE71698119017E014480068EF
:1025000003210840022804D1FFE748F2000011909F
:102510000BE00F48006803210840032803D1FFE7C0
:102520000A48119000E0FFE7FFE7FFE7FFE7119897
:10253000179000E0FFE717981CB0704706070809DE
:102540000102030400093D002C10024000127A0031
:1025500030100240003FAB01809FD50081B00146A2
:102560006846018000881F220146114001238B40EC
:102570008109494A88581843885001B07047C046BD
:1025800081B001466846018000881F220146114043
:1025900001238B408109404A88589843885001B0F4
:1025A0007047C04681B001466846018000881F22FE
:1025B0000146114001238B408109374A885818434E
:1025C000885001B07047C04684B00020039002904C
:1025D00031490868012210430860FFE70398401C56
:1025E00003902D480068022108400290FFE70299FD
:1025F0000020019041B9FFE7039840F20051401AD2
:10260000411E88410190FFE70198C0070028E5D1ED
:10261000FFE7214800688007002802D4FFE7FFE7B2
:10262000FEE71E49086807229043086008680222F6
:10263000104308601A49009108680860086808603B
:10264000086808600868174A104008600868164A59
:102650001043086010490868012212061043086000
:10266000FFE70D4800688001002801D4FFE7F8E784
:102670000B4908680322904308600868022210434F
:102680000860FFE7064800680007002801D4FFE75C
:10269000F8E704B07047C046001002400020024036
:1026A00004100240FFFFC2F70000040880B5FFF7E6
:1026B0008BFF80BD80B588B00790069140F2106016
:1026C000FFF74CFF9148019000F026F802A8009017
:1026D00000F05EF900990198069A0A8000228A802B
:1026E000079B0493CA8000F099F80198012100F03B
:1026F0001DF914200321FFF721FD019800F085F852
:1027000008B080BD82B001906846018000880199C0
:10271000486202B07047000080B58AB009900998FD
:1027200008907849884226D0FFE708982C498842CB
:1027300029D0FFE70898744988422CD0FFE7089811
:102740006F4988420FD0FFE70898704988422BD024
:10275000FFE708986E4988422FD0FFE708986D4937
:10276000884232D039E023480790FFF71BFF0798D3
:10277000FFF706FF32E01E480690FFF713FF0698AA
:10278000FFF7FEFE2AE019480590FFF70BFF0598BA
:10279000FFF7F6FE22E040F208400490FFF702FF48
:1027A0000498FFF7EDFE19E040F210300390FFF7B8
:1027B000F9FE0398FFF7E4FE10E00B480290FFF7E4
:1027C000F1FE0298FFF7DCFE08E006480190FFF7F3
:1027D000E9FE0198FFF7D4FE00E0FFE70AB080BDF4
:1027E0000010004012030000110300000404000068
:1027F000010400000B03000081B0009000990868FC
:1028000001229043086001B0704781B000900099A8
:10281000086801221043086001B0704782B001903F
:102820000091009800880199886201983449884293
:1028300005D0FFE701983349884212D1FFE701999B
:1028400008687022904308600098428801990868DF
:102850001043086000988288019908681043086056
:10286000FFE7009880680199C8620198244988426E
:1028700019D0FFE701982349884214D0FFE7019857
:10288000214988420FD0FFE70198204988420AD0A9
:10289000FFE701981E49884205D0FFE701981D49CE
:1028A00088420DD1FFE70199086840F20032904359
:1028B00008600098C2880199086810430860FFE723
:1028C00001980F4988420FD0FFE701980F498842CD
:1028D0000AD0FFE701980E49884205D0FFE701982A
:1028E0000C49884205D1FFE70098007B01990863F5
:1028F000FFE70199486901221043486102B070471F
:10290000002C014000040040002000400040014035
:10291000004401400048014082B001900091009ABB
:102920000199C8689043C86002B0704782B00190B6
:102930000091009A0199C8681043C86002B07047BE
:1029400082B001900091009A019908699043086152
:1029500002B0704784B0029001910298C06801995A
:1029600008400090029800690199084207D0FFE7EB
:10297000009820B1FFE703A90120087003E003A934
:1029800000200870FFE703A8007804B0704700003B
:1029900081B000900099002008800099488000993B
:1029A0008880009A034991600099C8800099087353
:1029B00001B07047FFFF000085B0049003A80180BC
:1029C00002A9FF20087001A90870FFE703AA108878
:1029D000411E1180A0B1FFE701A90878049A531C99
:1029E00004931278504000900298009B084AD25CF1
:1029F0005040087000990748405C02A90870E5E75C
:102A000002A80078000201A90978401805B07047B3
:102A1000CC340008CC35000880B588B0079006910A
:102A2000002005900490039002900798019041497E
:102A300088420AD0FFE70198E34988420AD1FFE7BC
:102A40000520FFF74FFC059005E00220FFF74AFC48
:102A5000059000E0FFE7079800680004002818D5FB
:102A6000FFE70598400006994A088018B0FBF1F08E
:102A70000290029813490840049002980007400F02
:102A8000039004A8008803A9098808430799C8602F
:102A900016E0059806994A088018B0FBF1F00290FC
:102AA000029808490840049002980F2108400390BA
:102AB00004A8008803A9098808430799C860FFE7AC
:102AC00008B080BDF0FF000081B000900098406A1F
:102AD0000649084001B0704782B00190009100980B
:102AE000024908400199886202B07047FF01000066
:102AF00080B584B00390039802900E4988420DD0AF
:102B0000FFE70298B049884210D1FFE70B480190D7
:102B1000FFF748FD0198FFF733FD08E006480090F5
:102B2000FFF740FD0098FFF72BFD00E0FFE704B042
:102B300080BDC04600440040110400000E030000A8
:102B400081B000900099086801221043086001B02C
:102B5000704782B001906846018000881F210840BC
:102B6000012282400199086A1043086202B070474E
:102B700084B0009101460098029101A90880029852
:102B80000A889209805809881F221140C840C0074E
:102B900020B1FFE703A90120087003E003A900208A
:102BA0000870FFE703A8007804B0704782B0019076
:102BB0006846018000881F220146114001238B4096
:102BC0000199820988589843885002B0704782B0B2
:102BD00001906846018000881F22014611400123B0
:102BE0008B400199820988581843885002B0704779
:102BF00082B00190009100980C49884208D1FFE70B
:102C00000199D022885848F20003984388500BE07D
:102C100000981F2109040840000C012282400199FC
:102C2000086A10430862FFE702B0704709340F34A6
:102C300010B585B003900291002001900090039898
:102C400002A9098889094058029C1F231C400121C0
:102C50000A46A240104001900398029A920D8058B3
:102C6000029A1B041A40120C9140084000900098F0
:102C700038B1FFE7019820B1FFE704A901200870EF
:102C800003E004A900200870FFE704A8007805B05D
:102C900010BD82B001900091019908680122904313
:102CA00008600199086840F2006290430860009A49
:102CB000019908681043086002B0704782B0019023
:102CC000009101990868042290430860009A0199D4
:102CD00008681043086002B0704782B0019000910C
:102CE000019908680122904308600199486843F2FD
:102CF000000290434860009A019948681043486078
:102D000002B0704782B001900091019908680822D2
:102D100090430860009A019908681043086002B067
:102D2000704782B001900091019908680122904398
:102D300008600199086841F2000290430860009A17
:102D4000019908681043086002B0704780B582B0EE
:102D5000024601A802706A461170007801280BD162
:102D6000FFE719480521FFF732FF0920C00640F6AA
:102D70000001FFF767F80AE013480521FFF716FF87
:102D80000920C00640F60001FFF764F8FFE7684637
:102D9000007801280BD1FFE70B480621FFF717FF4A
:102DA0000920C00640F60001FFF754F80AE0064883
:102DB0000621FFF7FBFE0920C00640F60001FFF7E1
:102DC00041F8FFE702B080BD0038014080B582B015
:102DD000144801900021FFF795FC01980121009112
:102DE000FFF7AEFD00990198FFF796FD0198FFF7F8
:102DF00003FD02B080BDC04680B582B00948019095
:102E00000021FFF77FFC019801210091FFF798FD59
:102E100000990198FFF78AFD0198FFF7F6FC02B0D0
:102E200080BDC0460020004010B586B005A9002036
:102E30000870B648007808B9FFE704E05048B24986
:102E4000E322FDF7CDF904A800F098F9AC4800782A
:102E5000029000287ED0FFE70298012804D0FFE707
:102E6000029802284ED086E0FFF7C6FF04A800783B
:102E70003A2806D1FFE7A849002008704149088098
:102E80003FE004A800780D2804D1FFE79C49022008
:102E9000087035E004A80078FFF7C4F903A90870AA
:102EA0009D480078019020B1FFE70198012817D0D4
:102EB00025E034480088FF280BDCFFE70398000179
:102EC000314909682F4A12888854934901200870B3
:102ED00015E08B4900200870FFF778FFFFE70EE050
:102EE000039C2948026827490B88D05C2043D054B2
:102EF0000888401C0880884900200870FFE7FFE729
:102F0000FFE738E004A800788149097888420BD1AE
:102F1000FFE7FFF75BFF7A4900200870012000F00F
:102F20001DF905A9087014E004A800783A280BD10F
:102F3000FFE7794900200870124908807049012094
:102F40000870FFF759FF03E06D4900200870FFE7A4
:102F5000FFE710E004A800783A280BD1FFE7FFF75D
:102F60004BFF0849002008806B4908706449012024
:102F70000870FFE7FFE705A8007806B010BDC0465F
:102F80004A3700087E0200200800002080B55C4817
:102F90000078401E012804D8FFE759490020087036
:102FA00011E057480078012805D0FFE75448007821
:102FB000022801D1FFE705E00548534940F2A71276
:102FC000FDF70EF9FFE7FFF701FF002080BDC046C7
:102FD000A037000880B588B007A9002008704848CD
:102FE000007808B9FFE705E04648474940F24F122C
:102FF000FDF7F6F845480078059004287BD8059938
:103000008A0001A08018874600F070B800F006B86A
:1030100000F011B800F050B800F056B806A83A21F8
:103020000170007800F028F93849022008703A4908
:10303000002008705FE037480088012834DBFFE794
:1030400035480078049020B1FFE70498012810D09B
:1030500029E03248006800780009FFF7B9F8014616
:1030600006A80170007800F007F92B4901200870CC
:1030700019E02A480390006800780F210840FFF704
:10308000A7F8014606A80170007800F0F5F803994A
:103090000868401C08602049002008701D49088805
:1030A000401E0880FFE706E00D2000F0E5F8174914
:1030B00003200870FFE71EE01548007800F0DCF8F8
:1030C00012490420087016E0104901910020029076
:1030D0000870032000F042F8029907AA107001203E
:1030E000FFF734FE01990298087004E001200021E6
:1030F000FFF72CFEFFE707A8007808B080BDC046A8
:103100001E0100202F370008E637000820010020AC
:1031100059010020A20200200E01002038010020E9
:1031200082B001906946002008701248007858B1BA
:10313000FFE711480078019908700E4900200870D7
:10314000694601200870FFE76846007802B07047C2
:1031500008490020087001207047C04681B06946C8
:1031600008700449012008700099034A117001B0E9
:103170007047C046A40200201C01002080B582B028
:1031800001904348FFF7A0FC01990870012002B0AC
:1031900080BDC04610B58CB00BAC20700A9109A858
:1031A000027008A803701B2000210591FEF7C6FFDE
:1031B0002F48FFF7D3F90920C0060390012107919A
:1031C00040F200220092FEF7DDFD009B0398079A73
:1031D00002210191FEF76DFE009B03980599079A65
:1031E000FEF7AEFE0398079940F200420292FEF706
:1031F000C9FD0199029B0398079AFEF75AFE029BAC
:1032000003980599079AFEF79BFE0398059A07997C
:1032100040F600030493FEF74CFE0398049B0599C7
:103220000322FEF78DFE1348FFF798F91848069021
:10323000FFF75EFC06980A99FFF7EEFB05990698E2
:10324000FFF74BFD05990698FFF76BFD059906986A
:10325000FFF71FFD06980421FFF730FD06980821AF
:10326000FFF750FD0698FFF76BFC07980CB010BDF8
:10327000110500000E06000080B582B0014601A8CD
:10328000017001780248FFF727FC012002B080BDE1
:103290000038014080B58AB009A90191088040F248
:1032A0000870FFF75BF912480390FFF735FA05A89D
:1032B0000290FFF76DFB019B029903980D4A0A806B
:1032C00000228A801B885B1E0793CA80FFF7A6FA3C
:1032D000039801210491FFF729FB04991320FEF7BD
:1032E0002DFF0398FFF791FA04980AB080BDC046FD
:1032F000002000400F0E000080B584B003A900201C
:1033000008706F48007808B9FFE704E023486B496C
:10331000F022FCF765FF02A8FFF730FF6548007850
:103320000190032835D801998A0001A080188746AA
:1033300000F006B800F00AB800F017B800F003B8C3
:10334000FFF75AFD25E0FFF757FD22E0144B002060
:10335000188002981A88511C1980124988545549BE
:1033600002200870FFF748FD13E00D480088FF2891
:1033700008DCFFE702980A4B1A88511C198009499A
:10338000885403E04B4903200870FFE7FFF734FD42
:10339000FFE703A8007804B080BDC0464A370008A4
:1033A0007C0200207A01002080B582B001A90020B3
:1033B000087040480078009040B1FFE7009802286C
:1033C0000AD0FFE7009803280CD00CE00020FFF79C
:1033D000C5FE01A908701CE00120FFF7BFFE01A98E
:1033E000087016E015E03348007850B1FFE7314827
:1033F0000078022805D0FFE72E480078032801D185
:10340000FFE705E007482D4940F26512FCF7E8FEAA
:10341000FFE7FFF7DBFC27490120087001A80078CF
:1034200002B080BDCC36000880B584B003A900206E
:10343000087020480078012801D1FFE705E01E4808
:103440001E4940F22B12FCF7CBFE1D48007802907B
:1034500020B1FFE70298012805D026E001200021D5
:10346000FFF774FC21E01748008878B1FFE71648A1
:10347000019000680078FFF7FFFE01990868401C82
:10348000086010490888401E08800DE00320FFF7FF
:1034900065FE03A90870012000210091FFF756FC8A
:1034A000009807490870FFE7FFE703A8007804B019
:1034B00080BDC0461D0100202F3700088A37000854
:1034C0001F010020A00200203401002000C1814023
:1034D00001C0804101C0804100C1814001C08041E4
:1034E00000C1814000C1814001C0804101C08041D4
:1034F00000C1814000C1814001C0804100C18140C4
:1035000001C0804101C0804100C1814001C08041B3
:1035100000C1814000C1814001C0804100C18140A3
:1035200001C0804101C0804100C1814000C1814093
:1035300001C0804101C0804100C1814001C0804183
:1035400000C1814000C1814001C0804101C0804173
:1035500000C1814000C1814001C0804100C1814063
:1035600001C0804101C0804100C1814000C1814053
:1035700001C0804101C0804100C1814001C0804143
:1035800000C1814000C1814001C0804100C1814033
:1035900001C0804101C0804100C1814001C0804123
:1035A00000C1814000C1814001C0804101C0804113
:1035B00000C1814000C1814001C0804100C1814003
:1035C00001C0804101C0804100C1814000C0C101F3
:1035D000C30302C2C60607C705C5C404CC0C0DCD83
:1035E0000FCFCE0E0ACACB0BC90908C8D81819D9F3
:1035F0001BDBDA1A1EDEDF1FDD1D1CDC14D4D51523
:10360000D71716D6D21213D311D1D010F03031F112
:1036100033F3F23236F6F737F53534F43CFCFD3D42
:10362000FF3F3EFEFA3A3BFB39F9F83828E8E92932
:10363000EB2B2AEAEE2E2FEF2DEDEC2CE42425E5E2
:1036400027E7E62622E2E323E12120E0A06061A152
:1036500063A3A26266A6A767A56564A46CACAD6D02
:10366000AF6F6EAEAA6A6BAB69A9A86878B8B97972
:10367000BB7B7ABABE7E7FBF7DBDBC7CB47475B5A2
:1036800077B7B67672B2B373B17170B05090915192
:103690009353529296565797559594549C5C5D9DC2
:1036A0005F9F9E5E5A9A9B5B9959589888484989B2
:1036B0004B8B8A4A4E8E8F4F8D4D4C8C4484854562
:1036C0008747468682424383418180402820655255
:1036D00063765374617465203D3D205354415445D5
:1036E0005F52585F494E49542029207C7C20282075
:1036F000655263765374617465203D3D2053544197
:1037000054455F52585F5243562029207C7C202824
:1037100020655263765374617465203D3D20535497
:103720004154455F52585F4552524F52202900651F
:103730005263765374617465203D3D205354415467
:10374000455F52585F49444C450065536E6453745D
:10375000617465203D3D2053544154455F54585F8A
:1037600049444C45007573526376427566666572CE
:10377000506F73203C204D425F5345525F5044557B
:103780005F53495A455F4D4158002E2E2F6D6F648F
:103790006275732F7274752F6D627274752E63006B
:1037A0002820655263765374617465203D3D205333
:1037B000544154455F52585F5243562029207C7C27
:1037C000202820655263765374617465203D3D2046
:1037D00053544154455F52585F574149545F454FD8
:1037E0004620290030002E2E2F6D6F646275732FD6
:1037F00061736369692F6D6261736369692E630028
:103800002038000800000020980000001001000887
:10381000B838000898000020100A00002C010008A9
:1038200000A24A04020000007A010020E803980880
:10383000D007000011000000AD11000804000000D6
:103840007F0F000803000000A90E00081000000010
:10385000DD130008060000008D12000817000000AC
:103860005910000801000000A90C00080500000024
:10387000DD1100080F000000F9120008020000002E
:10388000A90D00080000000000000000000000007A
:103890000000000000000000000000000000000028
:1038A0000000000000000000000000000000000018
:0838B000000000000000000010
:04000005080000CD22
:00000001FF
